:100000000C9458000C9480000C9480000C94800098
:100010000C9480000C9480000C9480000C94800060
:100020000C9480000C9480000C9480000C94800050
:100030000C9480000C9480000C9480000C94800040
:100040000C94E2020C9480000C9480000C948000CC
:100050000C9480000C9480000C9480000C94800020
:100060000C942C030C948000000000002500280054
:100070002B00040404040404040402020202020229
:10008000030303030303010204081020408001025C
:1000900004081020010204081020000000080002DB
:1000A00001000003040700000000000000004B04F2
:1000B00011241FBECFEFD8E0DEBFCDBF11E0A0E01E
:1000C000B1E0ECEBFBE002C005900D92A034B1076B
:1000D000D9F722E0A0E4B1E001C01D92A631B20739
:1000E000E1F710E0C8E5D0E004C02197FE010E94CE
:1000F000D605C735D107C9F70E946C040C94DC05FE
:100100000C94000090E0FC01E656FF4F2491FC01A6
:10011000EA57FF4F3491FC01EE58FF4FE491EE2374
:10012000B1F0222339F02330E9F090F4213001F1CD
:10013000223011F1F0E0EE0FFF1FE859FF4FA591BB
:10014000B4918FB7F894EC913E2B3C938FBF0895F8
:100150002730A9F02830C9F0243061F78091800061
:100160008F7D03C0809180008F7780938000E2CFE5
:1001700084B58F7784BDDECF84B58F7DFBCF809132
:10018000B0008F778093B000D5CF8091B0008F7D85
:10019000F9CF08950895AF92BF92CF92DF92EF9278
:1001A000FF920F931F93CF93DF936C017B018B0121
:1001B000040F151FEB015E01AE18BF08C017D10771
:1001C00059F06991D601ED91FC910190F081E02DFB
:1001D000C6010995892B79F7C501DF91CF911F9150
:1001E0000F91FF90EF90DF90CF90BF90AF90089568
:1001F0003FB7F8948091EA019091EB01A091EC0156
:10020000B091ED0126B5A89B05C02F3F19F00196CE
:10021000A11DB11D3FBFBA2FA92F982F8827BC0160
:10022000CD01620F711D811D911D42E0660F771F88
:10023000881F991F4A95D1F708958F929F92AF9288
:10024000BF92CF92DF92EF92FF924B015C010E942E
:10025000F8006B017C010E94F8006C197D098E0981
:100260009F09683E734081059105A8F321E0821A39
:100270009108A108B10888EEC80E83E0D81EE11CE1
:10028000F11C81149104A104B10429F7FF90EF90AF
:10029000DF90CF90BF90AF909F908F90089508957A
:1002A00085ED8093BC008091BC0084FDFCCF109252
:1002B000F401089520918001260F3327331F213246
:1002C0003105ECF42091F401FC0190E080E0243051
:1002D00069F082E00895A09180012191AC01405A1B
:1002E0005E4FA40FB52FB11D2C930196861798F37E
:1002F00080918001680F6093800180E0089581E023
:1003000008950895E091F8018091F701E81730F41D
:10031000F0E0E05CFE4F808190E008958FEF9FEF6A
:1003200008959091F8018091F7012FEF3FEF981712
:1003300048F4E92FF0E0E05CFE4F208130E09F5F61
:100340009093F801C90108958091F7019091F80107
:10035000891B990B0895CF92DF92EF92FF920F9332
:100360001F93CF93DF937C01CB018A012091C701BA
:10037000222389F0EB016B01C40ED51ECC15DD05DF
:1003800069F06991D701ED91FC910190F081E02D28
:10039000C7010995F3CF642F0E945A01C801DF916C
:1003A000CF911F910F91FF90EF90DF90CF90089524
:1003B000CF93DF931F92CDB7DEB769832091C7013A
:1003C0002223F9F02091F501203258F021E030E0AD
:1003D000FC013383228390E080E00F90DF91CF9186
:1003E00008958091F601E82FF0E0E853FE4F9981DF
:1003F00090838F5F8093F6018093F50181E090E018
:10040000ECCF61E0CE0101960E945A01F7CFCF9365
:10041000FC01C48121E02093C701C093E801109240
:10042000F6011092F5018485682B8DEF91E00E9412
:10043000D8019091F501913208F03FC08091F4010C
:100440008111FCCF82E08093F40181E08093F3017D
:100450008FEF8093C6011092C5019093C401A8EC60
:10046000B1E0E4EAF1E080E098132FC01092A3011C
:100470008091A301CC0FC82BC093A3018091F201FE
:10048000813039F51092F2018091A3018093BB0075
:100490008091BC0083FDF8CF85EC8093BC008091F7
:1004A000F4018230E1F38091C6018F3F31F08091F9
:1004B000C601803211F08091C6011092F6011092AF
:1004C000F5011092C701CF9108952D9121938F5F6F
:1004D000CBCF85EEE2CF90E080E00895FC01019063
:1004E0000020E9F73197AF01481B590BBC0189E0A7
:1004F00092E00C94CB000F931F93CF938C01C62FE7
:100500000E9407026C2F6460C8010E9407026C2FD2
:100510006B7FC8010E94070283EC90E00197F1F71E
:10052000CF911F910F9108950F931F93CF93DF9356
:100530008C01D62FC42F607F642B0E947B0280E148
:10054000D89FB00111246C2BC801DF91CF911F916E
:100550000F910C947B02CF93DF93CDB7DEB7289732
:100560000FB6F894DEBF0FBECDBF98E0E0E0F1E03B
:10057000DE01119601900D929A95E1F7909111028A
:10058000981708F48FEF90E0880F991F21E030E072
:100590002C0F3D1F820F931FFC016081606840E0BB
:1005A00089E092E028960FB6F894DEBF0FBECDBF6B
:1005B000DF91CF910C94940241E00E94940281E07B
:1005C00090E008951F920F920FB60F9211242F936F
:1005D0003F938F939F93AF93BF938091F901909135
:1005E000FA01A091FB01B091FC013091E90123E0F7
:1005F000230F2D3758F50196A11DB11D2093E90158
:100600008093F9019093FA01A093FB01B093FC0150
:100610008091EA019091EB01A091EC01B091ED0184
:100620000196A11DB11D8093EA019093EB01A09367
:10063000EC01B093ED01BF91AF919F918F913F91EC
:100640002F910F900FBE0F901F90189526E8230F43
:100650000296A11DB11DD2CF1F920F920FB60F921D
:1006600011242F933F934F935F936F937F938F93B7
:100670009F93AF93BF93EF93FF938091B900887FCF
:10068000803609F44AC0F0F5883209F4A7C018F59D
:10069000803109F49BC0B8F4882309F4F9C088308C
:1006A00009F494C0FF91EF91BF91AF919F918F9109
:1006B0007F916F915F914F913F912F910F900FBE5E
:1006C0000F901F901895883109F488C0803251F737
:1006D0008093C60114C0803409F49DC040F4803377
:1006E000B9F38833F9F68093C60185ECB0C0803544
:1006F00009F485C0883509F496C0883499F60E94BB
:100700005001D0CF883909F48CC038F5883729F0EA
:1007100050F4883611F0803729F683E08093F40195
:100720001092A20157C0883809F47BC0803919F0B3
:10073000803809F0B7CF8091A201803208F071C0F3
:10074000E091A20181E08E0F8093A2018091BB0015
:10075000F0E0EE57FE4F80833DC0803B39F0E0F47F
:10076000803A09F479C0883A09F09CCF84E08093FC
:10077000F4011092810110928001E091F001F0915A
:10078000F10109958091800181110FC081E0809372
:1007900080011092600109C0803C09F4A6CF883C1A
:1007A00009F4A3CF883B09F07DCFE091810181E07E
:1007B0008E0F80938101F0E0E05AFE4F808180939C
:1007C000BB00909181018091800129C08091A3019B
:1007D0008093BB0085EC8093BC0064CF9091C501F1
:1007E0008091C401981758F5E091C50181E08E0F02
:1007F0008093C501F0E0EC55FE4F8081E9CFE09198
:10080000C50181E08E0F8093C5018091BB00F0E0AF
:10081000EC55FE4F80839091C5018091C4019817DB
:10082000C8F285E8D8CFE091C50181E08E0F8093B2
:10083000C5018091BB00F0E0EC55FE4F80838091B4
:10084000F30181115CCF81E08093F20184EA80930F
:10085000BC001092F40126CF85EC8093BC0010926E
:10086000F4018091A201803230F4E091A201F0E025
:10087000EE57FE4F10826091A20170E0E091EE0110
:10088000F091EF0182E891E009951092A2010ACF60
:100890001092C60134CFEDEFF1E01382128288EEA0
:1008A00093E0A0E0B0E084839583A683B7838CE0D7
:1008B00091E091838083E9E0F2E0138212828EE17D
:1008C00091E09183808311868FE3848380E1828726
:1008D00082E0838714860895CF93DF93CDB7DEB788
:1008E000A1970FB6F894DEBF0FBECDBF789484B544
:1008F000826084BD84B5816084BD85B5826085BD1C
:1009000085B5816085BD80916E00816080936E00A9
:10091000109281008091810082608093810080919B
:10092000810081608093810080918000816080934C
:1009300080008091B10084608093B1008091B0000C
:1009400081608093B00080917A00846080937A0007
:1009500080917A00826080937A0080917A00816031
:1009600080937A0080917A00806880937A00109258
:10097000C1001092F8011092F7011092F601109246
:10098000F5011092F40181E08093F3011092F201DD
:1009900082E10E94820083E10E9482008091B9007E
:1009A0008E7F8093B9008091B9008D7F8093B900CC
:1009B00088E48093B80085E48093BC0089EC90E0E3
:1009C0009093F1018093F0018AEC90E09093EF0115
:1009D0008093EE0110920E0280911402823018F082
:1009E00098E090930E028093110262E370E080E041
:1009F00090E00E941D016091150289E092E00E9442
:100A0000070268EE73E080E090E00E941D0160E361
:100A100089E092E00E947B020BE416E4C801019792
:100A2000F1F760E389E092E00E947B02C801019740
:100A3000F1F760E389E092E00E947B0283E592E0B7
:100A40000197F1F760E289E092E00E947B026091F9
:100A50000E02606240E089E092E00E94940284E02D
:100A600080930F0240E06CE089E092E00E949402E3
:100A700040E061E089E092E00E9494028BE39FE114
:100A80000197F1F780911202882319F080E00E940B
:100A9000AB0282E08093100240E066E089E092E0E1
:100AA0000E94940240E062E089E092E00E94940299
:100AB0008BE39FE10197F1F788E08093150260E0F6
:100AC00089E092E00E94070280E00E94AB0286E289
:100AD00091E00E946E0288EEC82E83E0D82EE12CB1
:100AE000F12C9AE0492E512C612C712C20E0A22E81
:100AF00020E0B22E81E00E94AB022FB7F894609103
:100B0000F9017091FA018091FB019091FC012FBFD6
:100B1000A70196010E94B40519A28E010F5D1F4F17
:100B2000CA01B901A30192010E94B405605DF801F8
:100B300062938F01211531054105510589F73097E1
:100B400019F0CF010E946E0286E391E00E946E02CE
:100B500064E670E080E090E00E941D01A114B10401
:100B600049F20E940000C6CFA1E21A2EAA1BBB1BAD
:100B7000FD010DC0AA1FBB1FEE1FFF1FA217B30769
:100B8000E407F50720F0A21BB30BE40BF50B661F7F
:100B9000771F881F991F1A9469F760957095809543
:100BA00090959B01AC01BD01CF010895EE0FFF1F91
:0C0BB0000590F491E02D0994F894FFCF1B
:100BBC00000040001400540000000000D801AB01FC
:100BCC006B028101A4019101820100000000DC0292
:100BDC00CB006B024F015669766120736F73696F9E
:100BEC00206C6F6B6F0020536567756E646F7300BC
:00000001FF
